:100000002728A301A200FF30A207031CA307031C9B
:1000100023280330A100DF300F200328A101E83E90
:10002000A000A109FC30031C1828A00703181528FC
:10003000A0070000A10F152820181E28A01C2228A8
:100040000000222808008313831203130800830191
:1000500007309900163083168500831285018030A1
:10006000831681008312A4010510851C39284428B9
:100070003C2885183C285B20051D4028542843282F
:10008000051943285B2035280514051E5328A40AAA
:100090000130A300F430022005302402031D532850
:1000A0000510A4013528442805140B30A300B830EE
:0C00B000022005103528051008005D280E
:02400E00C43FAD
:00000001FF
